:020000040000FA
:020000000C28CA
:080008008B01831618308500FE
:1000100083122C3085000B288316DF3081001830C6
:10002000850000308C0003308E0000308F000030DF
:100030009500003096002030990000309C00383048
:100040009F008312003081002F30850000308A002D
:1000500000308B0000308C000030900000309200A7
:1000600000309500173098000730990002309A0050
:100070000C309F00A001A101A201A301A401A501D0
:100080002F30A000432864002F30A0009F20A10043
:10009000AF2022082102031C6D2823082102031926
:1000A000532803186D28A50A25087F3C0318432808
:1000B000A501FE30AF202F30A0002108143C031C06
:1000C00066281430A300A2017D286D282208133C65
:1000D000031C6C281430A2008F280310210CA400EC
:1000E000A40A0310240C2102A20024082107A30063
:1000F000133C0318A201A501432864009F20143C6F
:10010000031C4328831608308104F83081058312CC
:100110002F30A00085006400630000007D2864008B
:100120009F2022020318432883160F308104831274
:100130002F30A00085006400630000008F281F148A
:10014000073085000230E4209F109F149F18A628D6
:100150001E08A400200885001F1024080800A40021
:100160000730A0042408FF3A031DB8280730DD2813
:100170002408FE3A031DBE280030DD282408FD3A7D
:10018000031DC4280430DD282408503C0318CA2865
:100190000630DD2824082D3C0318D0280230DD2845
:1001A00024081E3C0318D6280330DD282408143CFC
:1001B0000318DC280130DD280530F838A0052008B8
:1001C00085000530E420080064000B1DE4280B11B5
:0801D000FF3E031DE4280800B6
:02400E00EC00C4
:00000001FF
